:100000000204613200000000000000320000000025
:10001000000000320000000000000032000000007C
:100020000000003200000000000000000000C39546
:10003000F02212002E60044002E422740122120316
:100040008860044002E4227401220200591200591F
:1000500060044002E422740122C3EDB50706ECB54A
:100060000602E422740122780F790BE766A2E750BA
:1000700006E7A2E774FF22E50BB50F12E50AB50EFD
:100080000DE509B50D08E508B50C03C3E42274FFBE
:100090002212006760044002E422740122EAC39441
:1000A00008400408A380F72409FA2213DAFD22D3BA
:1000B000E433DAFDFAF4FB22AE02E6F70809DEFAD1
:1000C00022209802E4223098FDE599C29822C204C9
:1000D0008002D204120116B408061201291880F415
:1000E000200405B4200280EC300213C0E0C3946108
:1000F000400A941A5006D0E0545F8002D0E02003FA
:1001000003120129B40D0B200305740A120129E41E
:10011000F622F60880BE3098FDE599C29822740D4B
:10012000120129740A120129223099FDC299F59908
:10013000220022D2B53131D2B431317F0AD330B569
:100140000C30B409DFF8C2B43131C2B5C392042215
:10015000C2B43131D2B53131D2B42292B43131503E
:100160000C7F0A20B407DFFBD2B5D38013D2B531A0
:10017000317F0A20B507DFFBD2B4D38003C2B5C3F9
:1001800022D2B43131D2B531317F0A20B505DFFB3F
:10019000D38007A2B492D5C2B5C3227E0833315BA7
:1001A000400CDEF931814006A2D550023150920454
:1001B0002233FD7E083181400CA2D533DEF7CD130A
:1001C000CD315BD2B4920422F8745A0400000000CE
:1001D0000000000070F500D8F022C3AE02E637F749
:1001E0000809DEF9227408C0F08502F0A4FFD0F0FF
:1001F00078105108C37810511078085110500678C3
:100200000C791031DADFED22AE02760008DEFB2237
:10021000AE02E633F608DEFA22780C51082001110E
:10022000C2D574082A14F8E630E706B2D57808512A
:100230009420010F74102A14F8E630E706B2D5783E
:100240001051947810790875F008EAA4FBE626F6B8
:10025000C0D0BA0104D0D0800BD0D0AE021E08E6C8
:1002600033F6DEFA780CAE02E633F608DEFAAE02BA
:10027000780CE6970908DEFA19781040127908C35D
:10028000780CAE02E697F60908DEF97810190679BF
:1002900008DBBA22AE02D3E6F43400F608DEF82218
:1002A000C00179101200B8D001C00174102A14F8EE
:1002B000E6C0E0780851087808760AE9240FF9E4E6
:1002C000F719C0015119780CD001E62430F77810E5
:1002D000AE02E44608DEFC70E8D0E020010730E71B
:1002E00004742D19F7A801D0017A1012037322E5C6
:1002F0008104F5F02AF581C2D578105108A8F05193
:1003000008E76032B42D04D2D580289430C0E0C014
:10031000017810790C1200B8780851087808760A2C
:1003200031E5D001A8F0D0E0F6C001A8F079103195
:10033000DAD0010980CB30D50478105194E5F0145F
:10034000F58122C001C000782186040886057E8DD3
:100350007F351203A67E197F3612039F7821A604EB
:1003600008A605D006D007D20112043A85040885F4
:10037000050922E6F760040809DAF8E4F722E660E6
:10038000061201290880F722ED6FA2E75006EDA2C0
:10039000E774FF22C3EC9EFCED9FFDA2E74C22EC2C
:1003A0002EFCED3FFD221203C5EC8EF0A4F8A9F05F
:1003B000EC8FF0A429F9ED8EF0A429FDAC0030D526
:1003C000031203EA22C2D5C004C005AC06AD07ED96
:1003D00030E709B2D51203EAAE04AF05D005D00468
:1003E000ED30E705B2D51203EA22EDF4FDECF4247A
:1003F00001FC50010D2275F010E4F8F9FAFBC3EC92
:1004000033FCED33FDEA33FAEB33FBC3EA9EF582AE
:10041000EB9F4003FBAA82B3E833F8E933F9D5F048
:10042000DDC3222001031203C51203F6AC00AD01A7
:1004300020010630D5031203EA228D832001031226
:1004400003C51203F6AC02AD03E58320010630E7D5
:10045000031203EA22E62401F6FA08E63400F64A1B
:1004600022787FE4F6D8FD75814FC28E759852755B
:100470008922758DFDD28E75200074021201C8127A
:10048000054B120CA87841E6A2E750030204B2D251
:1004900005754803754900753E14753F00120656F0
:1004A000754803754900753EFA753F00120A6502EA
:1004B00004BDC205854138853840120558020482C2
:1004C00075420A754300780BE8836006120129081B
:1004D00080F60204EF736365676C69206C612076B7
:1004E000657273696F6E6520302C312C323A0012C0
:1004F000011E78231200CE79237A021202EF79428C
:1005000078101200B8AC42AD437E007F0012004A62
:10051000600302051B120656020544AC42AD437E41
:10052000017F0012004A60030205311208790205BA
:1005300044AC42AD437E027F0012004A60030205D4
:1005400044120A650204C0C2AF80FE7538FF7539D7
:100550000085384012055822120133744012019B65
:1005600074FF12019BE54012019B1201502275425B
:1005700001754300AC42AD437E087F0012004D7010
:10058000030205D775F001E54055F0C0E0784CD086
:10059000E0F6E54CB4000280030205B3780BE88373
:1005A00060061201290880F60205B0204F6E200077
:1005B0000205C7780BE88360061201290880F6025D
:1005C00005C7204F6666007840E6C313F6784212EE
:1005D00004556003020574740A120129740D120196
:1005E0002922AC4DAD4E7EFF7F0012003E6003021B
:1005F0000650AC4DAD4E7EFF7F0012043A8C468D06
:1006000047E5461201C8AC4DAD4E7EFF7F00120497
:10061000238C468D47754500854508750900750A88
:1006200000750B0085460C85470DE5477F0030E7D8
:10063000027FFF8F0E8F0F120091700302064D7420
:10064000FF1201C80545E54560030206180206557C
:10065000E54D1201C822AC48AD497EE87F03120384
:10066000A68C488D49853E3A853F3B754A00754BBF
:1006700000780BE88360061201290880F60206A6BE
:100680002876657273696F6E653029205620706513
:1006900072207661726961726520544320617474BE
:1006A00075616C653A0012011E783A7A027923125C
:1006B00002A0782312037E12011E786479001203CF
:1006C00043850845E545B44B02800250030206D637
:1006D000754503020709E545B43202800250030262
:1006E00006E8754502020709E545B4190280025083
:1006F000030206FA754501020709E545B4000280C8
:1007000002500302070975450085454475F003E56D
:10071000441200327003020765AA44783812009D23
:100720001200AFE65BF6853840120558853A4D85D4
:100730003B4E1205E2D39204AA4412009DE5381202
:1007400000AFE5382004035B80014AF53885384066
:10075000120558853A4D853B4E1205E20544E544A5
:10076000600302070C7A04E5380A1200ABB3920466
:100770007A0412009DE5381200AFE5382004035BCF
:1007800080014AF53878421200C1F6E408F6AC421E
:10079000AD437E767F0012004A60030207A3740116
:1007A0000207A4E4C0E0AC42AD437E567F001200D5
:1007B0004A60030207BB74010207BCE4D0F045F0B5
:1007C000B40102800302084D780BE8836006120131
:1007D000290880F60207EB496E732E206E756F763E
:1007E0006F2076616C6F72653A200078231200CE1C
:1007F00079237A021202EF793A78101200B8780B56
:10080000E88360061201290880F60208332876651D
:100810007273696F6E65203029562070657220767C
:100820006172696172652054432061747475616CF2
:10083000653A0012011E783A7A0279231202A078F2
:100840002312037E12011E754200754300AC3AADBF
:100850003BAE4AAF4B12039F8C4A8D4BA2059204CC
:100860005003020868020878AC4AAD4BAE48AF4965
:1008700012003E60030206BA22753AC8753B00AC0E
:100880003AAD3B7E027F001204238C3C8D3D780BF9
:10089000E88360061201290880F60208B756207026
:1008A00065722076617269617265205443206174BB
:1008B0007475616C653A0012011E783A7A027923E8
:1008C0001202A0782312037E12011E7864790012AE
:1008D0000343850845E545B44B02800250030208F6
:1008E000E775450302091AE545B432028002500358
:1008F0000208F975450202091AE545B41902800299
:10090000500302090B75450102091AE545B40002BE
:100910008002500302091A75450085454475F003AD
:10092000E5441200327003020976AA4478381200B6
:100930009D1200AFE65BF6853840120558853A4DAA
:10094000853B4E1205E2D39204AA4412009DE5387D
:100950001200AFE5382004035B80014AF538853882
:1009600040120558853C4D853D4E1205E20544E593
:1009700044600302091D7A04E5380A1200ABB39201
:10098000047A0412009DE5381200AFE53820040314
:100990005B80014AF53878421200C1F6E408F6ACF3
:1009A00042AD437E767F0012004A60030209B474B0
:1009B000010209B5E4C0E0AC42AD437E567F0012AF
:1009C000004A60030209CC74010209CDE4D0F0456D
:1009D000F0B401028003020A61780BE8836006121A
:1009E00001290880F60209FC496E732E206E756F8E
:1009F000766F2076616C6F72653A20007823120062
:100A0000CE79237A021202EF793A78101200B8AC4C
:100A10003AAD3B7E027F001204238C3C8D3D780B67
:100A2000E88360061201290880F6020A4756207002
:100A30006572207661726961726520544320617429
:100A40007475616C653A0012011E783A7A02792356
:100A50001202A0782312037E12011E754200754314
:100A6000000208CB22AC48AD497EE87F031203A602
:100A70008C488D49853E3A853F3B754A00754B0051
:100A8000AC3AAD3B7E027F001204238C3C8D3D7856
:100A90000BE88360061201290880F6020AC4287652
:100AA000657273696F6E65203229562070657220F9
:100AB0007661726961726520544320617474756156
:100AC0006C653A0012011E783A7A0279231202A06C
:100AD000782312037E12011E786479001203438585
:100AE0000845E545B44B0280025003020AF47545FF
:100AF00003020B27E545B4320280025003020B06C5
:100B0000754502020B27E545B41902800250030225
:100B10000B18754501020B27E545B4000280025011
:100B200003020B27754500854544AA447838120016
:100B30009D1200AFE65BF6853840120558853A4DA8
:100B4000853B4E1205E2D39204AA4412009DE5387B
:100B50001200AFE5382004035B80014AF538853880
:100B600040120558853C4D853D4E1205E20539E59C
:100B700039B4030280025003020BA47539007A04D1
:100B8000E5380A1200ABB392047A0412009DE538EE
:100B90001200AFE5382004035B80014AF538853840
:100BA0004012055878421200C1F6E408F6AC42AD96
:100BB000437E767F0012004A6003020BC27401027A
:100BC0000BC3E4C0E0AC42AD437E567F0012004A46
:100BD0006003020BDA7401020BDBE4D0F045F0B4E1
:100BE00001028003020C7C780BE883600612012965
:100BF0000880F6020C0A496E732E206E756F766FB0
:100C00002076616C6F72653A200078231200CE79ED
:100C1000237A021202EF793A78101200B8AC3AAD9A
:100C20003B7E027F001204238C3C8D3D780BE883D1
:100C300060061201290880F6020C6228766572733C
:100C4000696F6E65203229205620706572207661AA
:100C500072696172652054432061747475616C65BA
:100C60003A0012011E783A7A0279231202A0782300
:100C700012037E12011E754200754300AC3AAD3B73
:100C8000AE4AAF4B12039F8C4A8D4BA20592045083
:100C900003020C97020CA7AC4AAD4BAE48AF491209
:100CA000003E6003020AD822D288D2A8D2AF744193
:100CB000120133D2E012019BD31201B1120150F59F
:100CC0004174051201C8C2AFC2A822000000000092
:00000001FF
